:020000040000FA
:0600000000308600072815
:08000800AD0A0B1109000313FE
:1000100083121030850007309900A0308B0000302B
:1000200083168C00C5308100003086000C308500BE
:100030008312203084008001840A041F1B280030B2
:10004000AB0018222130D623AE002430D623B100D5
:100050002230D623B800B3000230D623BE001E30B3
:10006000D623C0002330D623AC00AC182C150430A6
:10007000B5003C120613E82141205E20FF20262215
:100080003C282030B9001330A900043005052A06A9
:1000900003195028C520B90B53280430AA0641285B
:1000A0002A30A9004A28C520043005052A0603196C
:1000B0004328C520E120A90B532808002508A100EA
:1000C0002608A2002708A3002808A400A501A6016D
:1000D000A701A80125308400702078208020080026
:1000E0000830A900A320A620800DA90B7228C528DE
:1000F000840AA320A620800DA320A620800DC52859
:10010000840A0430A900A320A620800C840AA3201E
:10011000A620800CA90303198F2884038328800E4E
:100120008403800EC528043005052A060319B90A80
:1001300008002A1D9F28C520051D9B280800C520F2
:1001400005199F2808002A199F289B28AD01C52062
:10015000043005052A060319B028AD18BE28A728C3
:10016000C520C520C520B9019320C520C5209320F6
:10017000C520E12093200230390208002030C2005F
:100180002F08C100C023992022282B18D4288512BB
:10019000010C7F390319D0282F02031C8510080099
:1001A000AF08031D851408008510010C7F39031961
:1001B000DD282F02031C85120800AF08031D8516D9
:1001C0000800BC1CFC2832082F02031CFA2803106C
:1001D0003B0D2C1C3B08323E2C180A3EA000010CA3
:1001E000A0020318C5287D3C031CF8280613C52867
:1001F0000617C5280617C528AC180613C5282108F8
:100200002502031D1F2922082602031D1F2923087A
:100210002702031D1F2924082802031D1F29210866
:100220002E02031919292C1F1F2921083102031D31
:100230001F29C520230824020319AC2920290800FE
:100240003C162808FE3E03194729FF3E03190513F3
:10025000FF3E03198613FF3E03194D29FF3E031984
:100260009821FF3E03197D21FD3E03195229FF3ECF
:1002700003190517FF3E03198617FF3E03194A2984
:10028000FF3E0319A221FF3E03198B21C629230833
:10029000073C71292308F83E71292308073C0318FD
:1002A0006529712908302702031C712903191F29A8
:1002B000FD3E03190517FF3E03198617FE3E03197D
:1002C000A221FF3E03198B21C62903197D21FF3E80
:1002D00003199821FE3E03198613FF3E03190513E7
:1002E000C629240801392B060319C6292408013917
:1002F000AB0020220130A300C629AC1E8929BC1EF8
:100300000800B9002230D623B800B300BC12390867
:10031000080086130800AC1E9629BC1A0800B90014
:100320000130B800B300BC16390808008617080071
:100330002C1DA029AC1C9E29BC1008003C110800F3
:10034000061308002C1DAA29AC1CA829BC140800FF
:100350003C15080006170800C5202308013A031DB4
:10036000C1293C18B729FF30B4000430B5003C184F
:100370006C223C18C6293C14AB090130AB05202285
:10038000C629AC18BC143C1CC6293C10C520E82169
:100390002308013A0319E5292308BB003C19DD298C
:1003A0000310BB0DAC1FE129A2080319E129221C8F
:1003B000BB0AA218E129BB0AE1293C1EE129303021
:1003C000BB073B08D623B2000800B201AF0108000A
:1003D0002C1A0A2A2B18FB2905120514AF08031939
:1003E0000510AC1D05143C1A0800A218F9290513C4
:1003F00008000517080005100516AF0803190512B7
:10040000AC1D05163C1A0800A218082A861308001D
:10041000861708002B18122A0512A2180514A21C10
:10042000051008000510A2180516A21C05120800E8
:100430002030D623AF00B2002530D623AB00080011
:100440002530C2002B08C100C02308003808013C39
:10045000031D2D2A3208AF00C5283C1232082F0296
:100460000319C528B30BC5283E082F020318412ADB
:10047000B20803193E2A3E08AF00412AAF01B30A71
:10048000C52832082F02031C472AAF03482AAF0AA7
:100490003808B300AD012630D623C5202F08BF0091
:1004A000C10B532A572ABF070318AD0A502A04303C
:1004B000C100C520AD0CBF0CAD13C10B592AAD084E
:1004C0000318642AAD0CBF0C2730D6233F08410225
:1004D000031C0030B307C528B40B0800702A0800BD
:1004E000FF30B400B50B0800A62AB600B60A0B30E0
:1004F000BC1BDC2BB60B7D2A080005140516DC237B
:1005000005100512DC237A2A0230B6002F30782A33
:1005100093222308013A0319882A93222308013AD7
:10052000031D8D2A080041205E2021082502031D9D
:10053000932A22082602031D932A23082702031D5B
:10054000932A24082802031D932A0800BC100930AE
:100550007522013075228822E223B9030319D72AB4
:10056000B9030319DF2AB9030319EA2AB9030319E6
:10057000242BB90303193A2BB90303194C2BB903E4
:100580000319542BB9030319662BB9030319792BEB
:10059000B90303198B2BB90303199E2B0430B9023D
:1005A0000319AC2B21080319B82B8422AB2A75221E
:1005B00088222130C2002108C100C023A92A752247
:1005C00088222230C200E2233908C1002230C20052
:1005D000C023A92A75228822E223C2000310C20D7B
:1005E00021080319092B10303902031CF92A84222F
:1005F000EB2A390875228822E2230310B90DB91FAE
:10060000032B8422FB2A3908C100C0230130752244
:10061000EB2A0630B600D623B900B6033603D6233C
:10062000B9020310390CC1073608C200C023831673
:100630009C18182B8312B60A1E3036020318A92AFA
:10064000B60AB60A36080B2B75228822E22304303C
:100650003902031C2D2B8422252B2330D623E7308F
:10066000C105B9033918C115B91841162330C200A4
:10067000C023A92A75228822E22303303902031CF1
:10068000432B84223B2B2330D623C112391CC116A5
:100690002330C200C023A92A752288222430C20038
:1006A0002108C100C023A92A75228822E223033031
:1006B0003902031C5D2B8422552B2330D623411392
:1006C000391C41172330C200C023A92A7522882271
:1006D000E22305303902031C6F2B8422672B233061
:1006E000D623F830C1053908C1042330C200C02325
:1006F000A92A75228822E22303303902031C822BA7
:1007000084227A2B2330D623C113391CC1172330FE
:10071000C200C023A92A75228822E22304303902AC
:10072000031C962B21303902031C982B84228C2B1E
:100730002630C2003908C100C023A92A75228822A8
:10074000E223B908031DA62B84229F2B2730C20069
:100750003908C100C023A92A8822E22303303902C4
:10076000031CB42B8422AC2BBC13391CBC17A92A44
:10077000FF30B4000430B5000130752290212228EA
:10078000410883169A008312420883169B008B133C
:100790001C129C111C1555309D00AA309D009C1404
:1007A0001C119C18D12B83128B17080083169B00F9
:1007B0001C141A0883120800AD01AD02AD08031D18
:1007C000DE2B0800B901A11FE82BB90A211FB90AC5
:1007D000A11EEE2B0330B907211EB907A11DF42B72
:1007E0000930B907211DB907A11CFA2B1B30B90725
:0807F000211CB90739080800BB
:02400E00C401EB
:104200000000000012000000140015001600180045
:104210001A001C001E0020002200250028002B0090
:104220002E00320036003A003E00430048004E00A7
:1042300054005A00600067006E0075007C000000AA
:1042400000002A000100A0002A00000010001E004B
:10425000000000000000000000000000000000005E
:104260000000000008000A000C000E001000120000
:10427000150018001B001E002100250029002D003C
:10428000FF00FF00FF00FF00FF00FF00FF00FF0036
:10429000FF00FF00FF00FF00FF00FF00FF00FF0026
:1042A000FF00FF00FF00FF00FF00FF00FF00FF0016
:1042B000FF00FF00FF00FF00FF00FF00FF00FF0006
:1042C000FF00FF00FF00FF00FF00FF00FF00FF00F6
:1042D000FF00FF00FF00FF00FF00FF00FF00FF00E6
:1042E000FF00FF00FF00FF00FF00FF00FF00FF00D6
:1042F000FF00FF00FF00FF00FF00FF00FF00FF00C6
:00000001FF
